:020000040000FA
:10000000831660308F000530810083128501073030
:100010009900831628309F00FA3085002230950021
:100020003F309200831293010C309500910112151C
:10003000203084008001840A841F1A282F30840015
:100040002C10AA010130AB00A020A8000339033A0C
:100050000319A8010F309F00AA0B2C289F182E28E7
:100060001E089F148C178C108C1871200B1D3428BF
:100070000B11B33081079F183B281E08A200BC203B
:10008000AB0B4D28AA0A0130AB002C1C4D282208CE
:100090002A0203182C102A08A20000009F14013025
:1000A000A80803195B281030A8180430A507031C02
:1000B0005C280508013A8500851E6028A4013328C4
:1000C0002408643A031D6C28A80A2808033A031977
:1000D000A80128089320AC14240A03193328A4008B
:1000E00033288C1085187728A001A1018428AB2023
:1000F000A000A106A100031D7F28AC1C0800AC10C5
:10010000A920120603399206200A03199028200E0E
:10011000150630399506A00C200C3F3993000800D5
:10012000FF30930008008C1F932883169A009B01D0
:100130001C1555309D00AA309D009C1483120800A8
:1001400083169B011C141A08831208008312920163
:10015000A628A90A0319A90100308A000310280D56
:100160008A070310220D03188A0AD43E03188A0A4C
:10017000290703188A0A82000008AD02031CAE0397
:1001800022088000AD070318AE0A840A373004063F
:100190002F30031984002E0CA3002D0CA200A30CF9
:1001A000A20CA30CA20C080000340034013400346B
:1001B0000234003403340034043400340534003491
:1001C0000634003407340034083400340934003471
:1001D0000A3400340B3400340C3400340D34003451
:1001E0000E3400340F340034103400341134003431
:1001F0001234003413340034143400341534003411
:1002000016340034173400341834003419340034F0
:100210001A3400341B3400341C3400341D340034D0
:100220001E3400341F3400342034003421340034B0
:100230002234003423340034243400342534003490
:100240002634003427340034283400342934003470
:100250002A3400342B3400342C3400342D34003450
:100260002E3400342F340034303400343134003430
:100270003234003433340034343400343534003410
:1002800036340034373400343834003439340034F0
:100290003A3400343B3400343C3400343D340034D0
:1002A0003E3400343F3400344034003441340034B0
:1002B0004234003443340034443400344534003490
:1002C0004634003447340034483400344934003470
:1002D0004A3400344B3400344C3400344D34003450
:1002E0004E3400344F340034503400345134003430
:1002F0005234003453340034543400345534003410
:1003000056340034573400345834003459340034EF
:100310005A3400345B3400345C3400345D340034CF
:100320005E3400345F3400346034003461340034AF
:10033000623400346334003464340034653400348F
:10034000663400346734003468340034693400346F
:100350006A3400346B3400346C3400346D3400344F
:100360006E3400346F34003470340034713400342F
:10037000723400347334003474340034753400340F
:1003800076340034773400347834003479340034EF
:100390007A3400347B3400347C3400347D340034CF
:1003A0007E3400347F3400348034003481340034AF
:1003B000823400348334003484340034853400348F
:1003C000863400348734003488340034893400346F
:1003D0008A3400348B3400348C3400348D3400344F
:1003E0008E3400348F34003490340034913400342F
:1003F000923400349334003494340034953400340F
:1004000096340034973400349834003499340034EE
:100410009A3400349B3400349C3400349D340034CE
:100420009E3400349F340034A0340034A1340034AE
:10043000A2340034A3340034A4340034A53400348E
:10044000A6340034A7340034A8340034A93400346E
:10045000AA340034AB340034AC340034AD3400344E
:10046000AE340034AF340034B0340034B13400342E
:10047000B2340034B3340034B4340034B53400340E
:10048000B6340034B7340034B8340034B9340034EE
:10049000BA340034BB340034BC340034BD340034CE
:1004A000BE340034BF340034C0340034C1340034AE
:1004B000C2340034C3340034C4340034C53400348E
:1004C000C6340034C7340034C8340034C93400346E
:1004D000CA340034CB340034CC340034CD3400344E
:1004E000CE340034CF340034D0340034D13400342E
:1004F000D2340034D3340034D4340034D53400340E
:10050000D6340034D7340034D8340034D9340034ED
:10051000DA340034DB340034DC340034DD340034CD
:10052000DE340034DF340034E0340034E1340034AD
:10053000E2340034E3340034E4340034E53400348D
:10054000E6340034E7340034E8340034E93400346D
:10055000EA340034EB340034EC340034ED3400344D
:10056000EE340034EF340034F0340034F13400342D
:10057000F2340034F3340034F4340034F53400340D
:10058000F6340034F7340034F8340034F9340034ED
:10059000FA340034FB340034FC340034FD340034CD
:1005A000FE340034FF3400340034013401340134AB
:1005B0000234013403340134043401340534013489
:1005C0000634013407340134083401340934013469
:1005D0000A3401340B3401340C3401340D34013449
:1005E0000E3401340F340134103401341134013429
:1005F0001234013413340134143401341534013409
:1006000016340134173401341834013419340134E8
:100610001A3401341B3401341C3401341D340134C8
:100620001E3401341F3401342034013421340134A8
:100630002234013423340134243401342534013488
:100640002634013427340134283401342934013468
:100650002A3401342B3401342C3401342D34013448
:100660002E3401342F340134303401343134013428
:100670003234013433340134343401343534013408
:1006800036340134373401343834013439340134E8
:100690003A3401343B3401343C3401343D340134C8
:1006A0003E3401343F3401344034013441340134A8
:1006B0004234013443340134443401344534013488
:1006C0004634013447340134483401344934013468
:1006D0004A3401344B3401344C3401344D34013448
:1006E0004E3401344F340134503401345134013428
:1006F0005234013453340134543401345534013408
:1007000056340134573401345834013459340134E7
:100710005A3401345B3401345C3401345D340134C7
:100720005E3401345F3401346034013461340134A7
:100730006234013463340134643401346534013487
:100740006634013467340134683401346934013467
:100750006A3401346B3401346C3401346D34013447
:100760006E3401346F340134703401347134013427
:100770007234013473340134743401347534013407
:1007800076340134773401347834013479340134E7
:100790007A3401347B3401347C3401347D340134C7
:1007A0007E3401347F3401348034013481340134A7
:1007B0008234013483340134843401348534013487
:1007C0008634013487340134883401348934013467
:1007D0008A3401348B3401348C3401348D34013447
:1007E0008E3401348F340134903401349134013427
:1007F0009234013493340134943401349534013407
:1008000096340134973401349834013499340134E6
:100810009A3401349B3401349C3401349D340134C6
:100820009E3401349F340134A0340134A1340134A6
:10083000A2340134A3340134A4340134A534013486
:10084000A6340134A7340134A8340134A934013466
:10085000AA340134AB340134AC340134AD34013446
:10086000AE340134AF340134B0340134B134013426
:10087000B2340134B3340134B4340134B534013406
:10088000B6340134B7340134B8340134B9340134E6
:10089000BA340134BB340134BC340134BD340134C6
:1008A000BE340134BF340134C0340134C1340134A6
:1008B000C2340134C3340134C4340134C534013486
:1008C000C6340134C7340134C8340134C934013466
:1008D000CA340134CB340134CC340134CD34013446
:1008E000CE340134CF340134D0340134D134013426
:1008F000D2340134D3340134D4340134D534013406
:10090000D6340134D7340134D8340134D9340134E5
:10091000DA340134DB340134DC340134DD340134C5
:10092000DE340134DF340134E0340134E1340134A5
:10093000E2340134E3340134E4340134E534013485
:10094000E6340134E7340134E8340134E934013465
:10095000EA340134EB340134EC340134ED34013445
:10096000EE340134EF340134F0340134F134013425
:10097000F2340134F3340134F4340134F534013405
:10098000F6340134F7340134F8340134F9340134E5
:10099000FA340134FB340134FC340134FD340134C5
:1009A000FE340134FF3401340034023401340234A3
:1009B0000234023403340234043402340534023481
:1009C0000634023407340234083402340934023461
:1009D0000A3402340B3402340C3402340D34023441
:1009E0000E3402340F340234103402341134023421
:1009F0001234023413340234143402341534023401
:100A000016340234173402341834023419340234E0
:100A10001A3402341B3402341C3402341D340234C0
:100A20001E3402341F3402342034023421340234A0
:100A30002234023423340234243402342534023480
:100A40002634023427340234283402342934023460
:100A50002A3402342B3402342C3402342D34023440
:100A60002E3402342F340234303402343134023420
:100A70003234023433340234343402343534023400
:100A800036340234373402343834023439340234E0
:100A90003A3402343B3402343C3402343D340234C0
:100AA0003E3402343F3402344034023441340234A0
:100AB0004234023443340234443402344534023480
:100AC0004634023447340234483402344934023460
:100AD0004A3402344B3402344C3402344D34023440
:100AE0004E3402344F340234503402345134023420
:100AF0005234023453340234543402345534023400
:100B000056340234573402345834023459340234DF
:100B10005A3402345B3402345C3402345D340234BF
:100B20005E3402345F34023460340234613402349F
:100B3000623402346334023464340234653402347F
:100B4000663402346734023468340234693402345F
:100B50006A3402346B3402346C3402346D3402343F
:100B60006E3402346F34023470340234713402341F
:100B700072340234733402347434023475340234FF
:100B800076340234773402347834023479340234DF
:100B90007A3402347B3402347C3402347D340234BF
:100BA0007E3402347F34023480340234813402349F
:100BB000823402348334023484340234853402347F
:100BC000863402348734023488340234893402345F
:100BD0008A3402348B3402348C3402348D3402343F
:100BE0008E3402348F34023490340234913402341F
:100BF00092340234933402349434023495340234FF
:100C000096340234973402349834023499340234DE
:100C10009A3402349B3402349C3402349D340234BE
:100C20009E3402349F340234A0340234A13402349E
:100C3000A2340234A3340234A4340234A53402347E
:100C4000A6340234A7340234A8340234A93402345E
:100C5000AA340234AB340234AC340234AD3402343E
:100C6000AE340234AF340234B0340234B13402341E
:100C7000B2340234B3340234B4340234B5340234FE
:100C8000B6340234B7340234B8340234B9340234DE
:100C9000BA340234BB340234BC340234BD340234BE
:100CA000BE340234BF340234C0340234C13402349E
:100CB000C2340234C3340234C4340234C53402347E
:100CC000C6340234C7340234C8340234C93402345E
:100CD000CA340234CB340234CC340234CD3402343E
:100CE000CE340234CF340234D0340234D13402341E
:100CF000D2340234D3340234D4340234D5340234FE
:100D0000D6340234D7340234D8340234D9340234DD
:100D1000DA340234DB340234DC340234DD340234BD
:100D2000DE340234DF340234E0340234E13402349D
:100D3000E2340234E3340234E4340234E53402347D
:100D4000E6340234E7340234E8340234E93402345D
:100D5000EA340234EB340234EC340234ED3402343D
:100D6000EE340234EF340234F0340234F13402341D
:100D7000F2340234F3340234F4340234F5340234FD
:100D8000F6340234F7340234F8340234F9340234DD
:100D9000FA340234FB340234FC340234FD340234BD
:100DA000FE340234FF3402340034003400340034A2
:100DB0000034003400340034003400340034003493
:100DC0000034003400340034003400340034003483
:100DD0000034003400340034003400340034003473
:100DE0000034003400340034003400340034003463
:02400E00C433B9
:10421000200068007400740070003A002F002F0026
:10422000700069006300700072006F006A00650032
:104230006300740073002E006F00720067002E0090
:1042400075006B00200020005000650074006500C0
:104250002000470072006900660066006900740073
:10426000680073002000280063002900200032004D
:104270003000300038002D003200300031003800AE
:1042800020002000500057004D0020004D006F001E
:1042900074006F007200200043006F006E00740015
:1042A00072006F006C006C006500720020007700E7
:1042B0006900740068002000720065006D006100F4
:1042C0007000200031002E0030002E003800200049
:1042D00043006F006D006D006F006E0020006300F2
:1042E0006F006400650020006200610073006500DB
:00000001FF
